:03000000021105E5
:03000B000200A54B
:03002B000202AE20
:03005B0002045F3D
:030073000204394B
:1000800002030406080C10182030406080040608A3
:100090000C10182030406080A0C00D0D0403060D28
:1000A0000503030202C2AFC0D0C0E020620C20688A
:1000B00002419D306602415DE47385258AC262E596
:1000C00025F4700221242068022111207210758B02
:1000D00000D0E0D0D0D292D291D290D2AF32D29290
:1000E000D291D2907406D5E0FDE53C1420E21520B3
:1000F000E10D207D02D295307D02D293020121D202
:1001000094020121207D02D293307D02D29502011A
:1001100021758B00D0E0D0D0D292D291D290D2AFC4
:1001200032758B00D0E0D0D0D2AF32419DE5256052
:100130000A207D02C292307D02C290D291419DE59B
:10014000256002C291207D02D290307D02D2924180
:100150009DE525600A207D02C290307D02C292207A
:100160007D02D292307D02D290419D207D02C293C9
:10017000307D02C295207D02C295307D02C293740B
:1001800006D5E0FDE525600A207D02C292307D02A1
:10019000C290D291419D207D02C293307D02C295D2
:1001A000C2947406D5E0FDE525600A207D02C29266
:1001B000307D02C290D291419DC294207D02C293B3
:1001C000307D02C2957406D5E0FDE5256002C2913E
:1001D000207D02D290307D02D292419DC294207D3A
:1001E00002C295307D02C2937406D5E0FDE525601C
:1001F00002C291207D02D290307D02D292419D2098
:100200007D02C295307D02C293C2947406D5E0FD92
:10021000E525600A207D02C290307D02C292207DD9
:1002200002D292307D02D290419D207D02C2953053
:100230007D02C293207D02C293307D02C295740676
:10024000D5E0FDE525600A207D02C290307D02C226
:1002500092207D02D292307D02D290419D30723D3B
:10026000E53C20E21A20E129207D02C293307D0284
:10027000C295207D02C295307D02C29302029D206C
:10028000E1E6207D02C293307D02C295C294020253
:100290009DC294207D02C295307D02C293E525F473
:1002A000F58A758B00D262D0E0D0D0D2AF32C2AF27
:1002B000C2AD53E6EFC0D0C0E0D2D3D2AFC2CEE5DC
:1002C0002960072074461529610C78007900E580C3
:1002D000307E01F430E40278FF53DACF207E03430E
:1002E000DA20307E0343DA10C2D8C271E580307E56
:1002F00001F430E40279FFC3E89970CE30610375F0
:1003000029402074037529408859D270E52A600479
:10031000152A611C20740543DA01C2D820700261DD
:1003200044A859206102C270207402612D882230D5
:10033000690AC3E522955E4003855E227882B60491
:1003400003852224C3E52594404002D26420CF0CCB
:10035000D0E0D0D0C2D343E610D2AD32C2CF7802C3
:10036000E52960053074021529C3E559940140055B
:10037000755C006186755D00756400E55C2401F5BF
:100380005C5003755CFF7982B7020EE547601EC3BF
:10039000E522943240178546227982B7030FE5475C
:1003A000600BC3E52294324004798E8722C3E52393
:1003B000952260084004152361BC0523D8C8056454
:1003C000E56470021564D565647565017805C3E55B
:1003D0006495664058C3E564956750087801756573
:1003E000030203F0C3E56495685005780175650163
:1003F000C3E55F9524401F7982B704028122E54757
:10040000701485245FE56404600385666475650186
:1004100075233C02042DE55F285005755FFF81229E
:10042000F55FE55F047006755DFF7564FFD0E0D091
:10043000D0C2D343E610D2AD32C0D0C0E0C2AF5379
:10044000917F53E67FC260759100C3E49550F594A7
:10045000E49551F595759104D0E0D0D0D2AF32C279
:10046000AF53E6EFC2ADC0D0C0E0C0F0D2D3D2AF40
:0E047000A8FBA9FCC2D830710281C653DACFB6
:10047E00207E0343DA10307E0343DA20D271E5800A
:10048E00307E01F420E402819D88268927C19D5388
:10049E00DACF207E0343DA20307E0343DA10C2D84F
:1004AE00C271307402C1897800E580307E01F4306B
:1004BE00E402C1898859C17053DACF207E0343DA32
:1004CE0020307E0343DA10C271206102A19653DA06
:1004DE00CF207E0343DA10307E0343DA20C2D8D217
:1004EE007188548955C3E89552F8E99553F9E4FBA0
:1004FE007E027A00C3E8948CE9940050057558008A
:10050E00A186C3E894C8E994005008E4D2E4FB7ACB
:10051E000AA163C3E89468E994015008E4D2E3FBAE
:10052E007A0FA163C3E894D0E994025008E4D2E2B2
:10053E00FB7A1EA163C3E894A0E994055008E4D2A7
:10054E00E1FB7A3CA163C3E89498E994085008E46F
:10055E00D2E0FB7A787E00C3E89556FCE99557FD0C
:10056E0030E708ECF42401FCEDF4FD755800C3EC03
:10057E009AED9E500375580188568957A854A9556F
:10058E00885289537802C170C3E89526F8E99527F9
:10059E00F9307C02C154307B02C154307A02C14D15
:1005AE00207502A1B9E9FDE8FCA1D8E9C313F9E869
:1005BE0013F8307902C14DE9C313F9E813F8307816
:1005CE0002C14DE9C313FDE813FC206126C3EC9470
:1005DE001CED94024002A1EFED7018C3EC94C850CC
:1005EE00120528C3E528940A5002C189755900D214
:1005FE0070C189E528600215287400207F03789663
:10060E00E624FAFEE43400FFC3EC9EFCED9FFD50A1
:10061E000678007900C154C3EC94FFED94004006B7
:10062E0078FF7900C154EC856FF0A4C5F0A2F733C2
:10063E00F87900400302067078FF7900020670E92F
:10064E00C313F9E813F8307C0EE9600278FFC3E8B3
:10065E001338F8E43400F9C3E894FFE9940040023B
:10066E0078FF8859D270206102C189741FF4552F0A
:10067E004BF52FC274E42B7002D27475294030747E
:10068E000375290A306102C19D20740353DAFE7589
:10069E002A20307403752A0AD0F0D0E0D0D0C2D30D
:1006AE00D2AD43E6103279010206D279030206D2A8
:1006BE00790A0206D2791E0206D279640206D2792E
:1006CE00C80206D27817E4D5E0FDD8FAD9F6227A18
:1006DE00147B780206F97A107B8C0206F97A0D7B70
:1006EE00B40206F97A0B7BC80206F9AC2575250112
:1006FE007902B27DE4C294D5E0FDE5256002C29197
:10070E00D5E0FDD291D5E0FDD294D5E0FDE5256092
:10071E000A207D02C292307D02C290E570D5E0FDC6
:10072E00207D02D292307D02D2907496D5E0FDD912
:10073E00C1EAF8D5E0FDD8FBDBB1C2948C2522C30B
:10074E007C007D0075F00005F0EA33FAEB33FB50C8
:10075E00F6EB13FBEA13FAC3E9FFE8FEE89AF8E9B1
:10076E009BF95004EFF9EEF8B3EC33FCED33FDD505
:10077E00F0DFEDF9ECF822E889F08A20D2D4F8A95E
:10078E00F07B0030F70B7BFFF42401F8E9F4340022
:10079E00F9E88520F0A4ADF0F8E98520F0A4AFF0DB
:1007AE00FEED2EF974003FFA7C04C3EA13FAE91346
:1007BE00F9E813F8DCF48BF030F70AE8F42401F8CA
:1007CE00E9F43400F9E889F0C2D4F8A9F02278826D
:1007DE00B6040302087EC3E5599419401FE52D5453
:1007EE00067019E547703878057994E71460077834
:1007FE000A1460027812C3E53B984020E547600971
:10080E0085615F7564FF756501852224E4F53EF50B
:10081E003FF540F541F542F54702087E75470179EF
:10082E0094E7147013E523F43333F913F8E9540104
:10083E0004F9E854FE020872E714147014E523F468
:10084E00333333F913F8E9540304F9E854FC02087E
:10085E007AE523F433333333F913F8E954070404F8
:0E086E00F9E854F8C39440F8E99400F9883E84
:10087C00893F22E547603BC3E53B13F9E53A13F8A2
:10088C00C3E53E98F8E53F99F9500CC3E89480E92C
:10089C0094FF40160208BAC3E8947FE99400500311
:1008AC000208BA787F79000208BA788079FF884309
:1008BC00894422E5476058E5432540F8E544354135
:1008CC00F9854420E4300701F43542FA30E709C3D6
:1008DC00EA94F040150208FCC3EA940F5003020896
:1008EC00FC78FF79FF7A0F0208FC780079007AF027
:1008FC00C3E524955E5006E52460092115E54420E6
:10090C00E70D2115E54430E706884089418A4222EB
:10091C00E547700302098078A1E6FAC3E54333F892
:10092C00E54433F9120785E930E70BC3E89480E915
:10093C0094FF40132157C3E8947FE994005002219F
:10094C0057787F79002157788079FFE820E715C325
:10095C00E52398F84009C3E89401400302097E7826
:10096C000102097EE8F424012523F8400302097EE4
:10097C0078FF884522E54770030209E378A2E6FA7E
:10098C00A841A942120785E930E70CC3E89401E9B4
:10099C0094FF40160209BAC3E894FFE9940050038F
:1009AC000209BA78FF79000209BA780179FFE920C7
:1009BC00E715C3E54598F84009C3E89401400302E4
:1009CC0009E178000209E1E8F424012545F8400327
:1009DC000209E178FF88242278FFC264E52D5406D1
:1009EC00702FD264C3E53B940A4009C3E5259440BB
:1009FC005002C264E53B601974FF853BF084853777
:100A0C00F0A4F8C5F0600278FFC3E895615002A825
:100A1C00618860227883E6F520120F2175E8901228
:100A2C0006B475E890E5E820ECFBA8BDA9BE120F52
:100A3C00A1756BAF756C00C3740013FD74AF13FC20
:100A4C0074AF2CFC74003DFDECFAEDFBC3E89AE9A5
:100A5C009B4014E56B24AFF56BE56C3400F56CEA48
:100A6C002CFAEB3DFB80E5AE6BAF6CC3E56C13F978
:100A7C00E56B13F8C3E913F9E813F8E56B28F5698E
:100A8C00E56C39F56A7A03C3E913F9E813F8DAF778
:100A9C00AA201A7009756B00756C00020ABA1AEA62
:100AAC006008EE28FEEF39FFDAF88E6B8F6C22753A
:100ABC00E890227883E6FFE5E820ECF7A8BDA9BE14
:100ACC00056DC3E56D94084052756D00E9FA79A087
:100ADC00E76044EA7007E56E601B020AF5C3E8950F
:100AEC006E6010E56E5006600C14020B010460F988
:100AFC00020B01E56EF56EC39458401B755EC0C3C6
:100B0C0094044013755E80C39404400B755E40C31F
:100B1C0094044003755E0075BB0322EFC39401601F
:100B2C001BC3E894FFE994035012C3E8956BE99555
:100B3C006C5009E55E600C155E020B4FE55EF460CF
:100B4C0002055EA85EC3E524985002A824C3E8956C
:100B5C005F400AA85FE55FF46003855F5E8825E56A
:100B6C006DB4070375BB1022743279A387F0A4C54A
:100B7C00F0A2F733F8C3E8955E4002A85E8822889D
:100B8C00248825886122753A00753B7F2275C82020
:100B9C00A8CCA9CD75C824AA38AB3988388939C3F3
:100BAC00E89AF8E99BF9AA3AAB3BAC3AAD3B7E0428
:100BBC007F02C3EB940440021E1FC3EB9408400257
:100BCC001E1FC3ED13FDEC13FCDEF7C3EA9CFAEB1E
:100BDC009DFBEF6009C3E913F9E813F8DFF7EA2886
:100BEC00FAEB39FB8A3A8B3B400122753AFF753B95
:100BFC00FF2230600261FE854C50854D51D260431E
:100C0C00E680227892E6FFC3E535948240010FC35B
:100C1C00E53594A040010FC3EF940640027F057E9A
:100C2C00021E3072010EC3E53B940350060E0E30CB
:100C3C0072010EC3E53B940250060E0E3072010E8B
:100C4C00A93BA83A7A04C3E913F9E813F8DAF7C315
:100C5C00E89EF8E99400F94009C3E89402E994008D
:0F0C6C0050047802E4F9E9FBE8FAC3E913FDE864
:100C7B0013FC884C894DC3EF94036037EF20E00DD4
:100C8B00E82CF8E93DF9ECFAEDFB020CABE828F89F
:100C9B00E939F9C3E89402F8E99400F97A02E4FB24
:100CAB00C3EF9403400D8A4E8B4F884889498C4A79
:100CBB008D4B22884E894F8A488B498C4A8D4B220B
:100CCB0030600281CBD26043E680E52D540660276D
:100CDB00A83AA93BE53494085006E820E002A94D58
:100CEB00759100C3E498F594E499F595759104D248
:100CFB006053917F43E68022D265753D00752000DD
:100D0B00020D16D265753D00752040E52D54066029
:100D1B0002C265D2AF206005E53D60012278017A01
:100D2B0002C3E53B940540027802C3E53B940A40BD
:100D3B00027803C3E53B940F40027A0330690478D1
:100D4B001E7A01206007E53D6003D2AF22D2AF00CF
:100D5B0000C2AFC3E53BFB940F40027B0FEB0430AB
:100D6B0073012320620123F93069027982E58BC379
:100D7B009940D0053DEAFBE59BF45440B52004DBDC
:100D8B00F6A1B2206502A116C265759100AE3AAF0D
:100D9B003BC3E49EF594E49FF595759104D26053A3
:100DAB00917F43E680A116306502A116D895D2AF8C
:100DBB002230690B0534206016753400020DDA20E1
:100DCB00600D20650A206B07158115810215C7225E
:100DDB00A84EA94F75910053917FC3E498F594E405
:100DEB0099F595759104854850854951D26043E634
:100DFB00802278003064053065027801E53575F0A6
:100E0B0007A4F9E5F028F5F0E9A2F013A2F113A27B
:100E1B00F213F535C394785003753578C3E53595E2
:100E2B00364008D266D292D291D290306002C1364F
:100E3B00854A50854B51D26043E68022C2AFC293A4
:100E4B00C294C29530720B9001FF7406D5E0FD027F
:100E5B000E5D207D02D293307D02D295759F107569
:100E6B003C02020F9CC2AF207D02D290307D02D299
:100E7B00923072179001DCC294207D02C295307DB6
:100E8B0002C2937406D5E0FD020E9990013F3062C9
:100E9B0006E5256002C291207D03759F20307D03FE
:100EAB00759F00753C03020F9CC2AFC293C294C2E4
:100EBB009530720B9001B97406D5E0FD020ECA2075
:100ECB007D02D295307D02D293207D03759F003039
:100EDB007D03759F20753C04020F9CC2AFD29130ED
:100EEB007217900196207D02C293307D02C295C28B
:100EFB00947406D5E0FD020F0790012D30620EE5CC
:100F0B0025600A207D02C292307D02C290759F102F
:100F1B00753C05020F9CC2AFC293C294C29530724E
:100F2B000B90016B7406D5E0FD020F37D294207D38
:100F3B0003759F20307D03759F00753C06020F9C47
:100F4B00C2AF207D02D292307D02D29030721F90C0
:100F5B00022A207D02C293307D02C295207D02C2FF
:100F6B0095307D02C2937406D5E0FD020F7C900193
:100F7B005130620EE525600A207D02C290307D0261
:100F8B00C292207D03759F00307D03759F20753CB9
:100F9B0001C266D2AF2290012BD292D291D290C2D3
:100FAB0093C294C295C262227880760708760708AE
:100FBB0076010876040876FF0876FF08760908762E
:100FCB0002087601087601788C760108760008769F
:100FDB00B40876FF0876FF0876FF0876030876FFDD
:100FEB000876010876FF0876250876D0087678080B
:100FFB0076C80876040876FF08760108760008762E
:10100B007A08760A087601227887E6FFC272BF0358
:10101B0002D2727888C27DE630E102D27DC27E7840
:10102B0089E630E102D27EC3EF94026008758E012F
:10103B00D273021045758E00C273227880E614902D
:10104B0000809378A1F67881E6149000809378A2C3
:10105B00F6120FA1227886E61490008D9378A3F6F2
:0F106B00120FA122789FE6F8700108C3E89411D4
:10107A0040027811E82828F5662566256628F5676E
:10108A0025662828F56822789CE67536FF75370CA0
:10109A00B402067536A075370AB40306753682752A
:1010AA00370522227896E6FA7897E6FB307F047AAB
:1010BA00007BFFC3EB9AFCC3948250027C82756F5B
:1010CA0000056FEC856FF0A4C3E5F0948040F2222E
:1010DA00D27F11AE1206C37A007B007C101206B9C9
:1010EA00E5592AFA74003BFBDCF37C04C3EB13FBDF
:1010FA00EA13FADCF7FEC27F11AE22E5EF20E6031F
:10110A007520000520903FFFE520146006901DFF22
:10111A001460009304600375EF12C2D353D9BF75EC
:10112A0081C043FF801206B475EF0243B203E5B3F0
:10113A00240420E702F5B3120FA17580FF75A400FD
:10114A0075F1D475D4EF75908775A54075F2FF7562
:10115A00D5BF75A60175E24275DB4675EA02120F24
:10116A00B312160278988670C2AF1206CD1206DD47
:10117A001206C31206E41206C31206EB1206C312C3
:10118A0017251206CD1206CD1206C8C2AFE4F8F62C
:10119A00D8FD78C879C8308407D9FBD8F7021C0073
:1011AA00120FB3121602111311461160116F119129
:1011BA0011AD11AE78988670120FA1758850758995
:1011CA001275C82475910475D84075A82275B8029D
:1011DA0075E690759B80759D0075D10E75BC587526
:1011EA00BB0375BA1175E8801206B4D2AF120A2091
:1011FA0043DA01C2D8C2711206CD753001D2617BC1
:10120A00037A0CE55870067A0CDB0221951206C3A4
:10121A002070022195C270E559C3940240E3E52F7C
:10122A00541F855B5AF55BB55AD7DAD7C26153DAD0
:10123A00CF207E0343DA20307E0343DA10C2D8C2BD
:10124A0071C2757528001206C8307409C3E528945E
:10125A000A4002D2751206B978023074027800C3C5
:10126A00E5599840F0C2AF1206DD1206DD1206DD1E
:10127A00D2AF1206CD7546001206B9788CE6C39431
:10128A00015003021356E530C3940150030213566A
:10129A00207435C3E55994FF5003021356C2AF12A6
:1012AA0006F2D2AF1206C8C3E559940150EFC2AF95
:1012BA001206DD1206BE1206DDD2AF1206C8C3E55B
:1012CA005994FF40E90217AA7F05D27F11AE120690
:1012DA00C8C2AFC27F11AEAE59C3E559947FD2AF2F
:1012EA0040741206B4C2AF1206F2D2AFDFDC11DAD2
:1012FA00C3EE94057897F61206CD12164412172DEE
:10130A007F0AD27F11AE1206C8C2AFC27F11AEAE3B
:10131A0059C3E559947FD2AF50E61206B4C2AF1250
:10132A0006DD1206BE1206DDD2AFDFD611DAEE24D2
:10133A00057896F61206CD12164412175C1206C8E4
:10134A0011AEC3E55994FF40F40217AAC3E55995B3
:10135A004640038559461206C878017988E7B403DE
:10136A00027805C3E5599840024182C2AF1206F2DB
:10137A001206F21206F2D2AF1206CD753000E4F56B
:10138A0031F5320531E531F470390532789AE6786B
:10139A0019146012783214600D787D14600878FA96
:1013AA00146003753200C3E532984017153275315F
:1013BA00B478998670C2AF1206F2D2AF7898867066
:1013CA001206C81206BEE529700530740221957806
:1013DA00012074027806C3E5599840A71206C8E5A9
:1013EA002970022195C2AF120FA1E4F522F523F567
:1013FA0024F525D2AF78858662F53EF53FF540F5AE
:10140A0041F542F56DF547F52CF52DF535120B92A0
:10141A00756D0875BB101206B4120ABBE5E820EC1C
:10142A00FBA8BDA9BEE97001F8886E120ABF756DE6
:10143A000875BB107887E6FE760211137887EEF6F8
:10144A00C2AF755EFF120B7485225E85225F85220C
:10145A0060D2AF752201752401752501855D647519
:0F146A006501D268D269753400120F21120F4B41
:10147900120B92120B99120C0F021490120FA11158
:1014890013756D0075BB03120D0E120DBC120DDB29
:101499001207DC120DFD120E47120B99120BFE12E8
:1014A9000C0F120CCB120D03120DBC120DDB12081E
:1014B9007F1209E4120DFD120E70120B99120BFE28
:1014C900120C0F120CCB120D0E120DBC120DDB12E9
:1014D90008BF120DFD120EB4120B99120BFE120C5D
:1014E9000F120CCB120D03120DBC120DDB12091CCD
:1014F900120DFD120EE6120B99120BFE120C0F12B1
:101509000CCB120D0E120DBC120DDB120981120D3E
:10151900FD120F21120B99120BFE120C0F120CCB9C
:10152900120D03120ABB120DBC120DDB120ABF12F7
:101539000DFD120F4B120B99120BFE120C0F120C10
:10154900CB30692F206B2C85615E85615F855D6479
:1015590075650179327A0AC3E534994009C269D2BD
:101569006A8A3302157CC3E5599401400302149039
:101579000215C7306A1B206B18E533147004C26A60
:101589008185F533C3E5599401400302149002158E
:10159900C7C3E55C9401400985615F855D64756534
:1015A90001C3E55C94FA5016307404E529600FC351
:1015B900E53B78F0306B0278609850028190C2AFB9
:1015C900120FA17887E6FE760211137887EEF6E40A
:1015D900F522F523F524F525F562C268D2AF120686
:1015E900B4120FA1307406E52970022195788DE6B1
:1015F900C394014002415F6188901A0D7820121648
:1016090086E520B4A50CA3121686E520B45A030278
:101619001624120FB3121644021643901A03788047
:101629007B0A121686A308DBF9901A0F788C7B15B2
:10163900121686A308DBF9901A2422C2AF1216C526
:1016490012169F901A00740D12168BA374021216AB
:101659008BA3741312168B901A0378807B0A1216C7
:101669008AA308DBF9901A0F788C7B1512168AA3C6
:1016790008DBF91216D81216B6901A2422E493F64A
:1016890022E6438F01538FFD75EF0275B7A575B734
:10169900F1F0538FFE22438F02438F0175EF0275DC
:1016A900B7A575B7F1901A0DF0538FFC22901A0D5A
:1016B90074A5D18B901A0E745AD18B227A3079D0B5
:1016C9007820901A40D186E520F709A3DAF7227A23
:1016D9003079D0901A40E7D18B09A3DAF922AB719E
:1016E900A872BB01027980BB02027981BB0302792E
:1016F90082BB04027994BB05027983BB0602798611
:10170900BB07027992BB08027987BB0902799CBBA6
:101719000A027988BB0B027989E8F7227C0512064F
:10172900CDDCFB22C2AF1206DD1206E41206EB1273
:1017390006F21206BE1206DD1206E41206EB1206C6
:10174900F21206BE1206DD1206E41206EB1206F2CA
:10175900D2AF22C2AF1206F21206EB1206E412064B
:10176900DD1206BE1206F21206EB1206E41206DDBF
:101779001206BE1206F21206EB1206E41206DDD2BA
:10178900AF22AE71AF72C2AF1206DD1206DD1206CC
:10179900DD1206BEDEF21206F21206BEDFF8D2AF85
:1017A90022F12DF125F1257571017572017573000D
:1017B900F18B7C05AD591206CDC3ED955970F5C372
:1017C900E5599401400AC3E55994FF40320217E6EE
:1017D900D1E7D144F12DC2AF75EF12F125DCD50562
:1017E90073C3E5739403500280C6F1250572E57150
:1017F9001490009A93F808C3E57298500280AE12CB
:1018090017251217250571C3E571940C5002809AAA
:0E181900120FB3121644C2AF75EF121217254C
:101A00000D021307070104FFFF09020101A55A0196
:101A100000B4FFFFFF03FF01FF25D078C804FF01DA
:051A200000FF0A01FFB8
:101A400023484B696E673530412320202020202019
:101A500023424C48454C4923463333302320202031
:101A60002020202020202020202020202020202076
:101C0000C2AFC2D353D9BF7581C043B20343FF8073
:101C1000752438752503B1BF75EF0275E24043F1B5
:101C20001053A4EFD284780379E67C1075220075F6
:101C30002300901DCC7B0675249875250130840205
:101C4000813D208408D8FBD9F9DCF781AD308408C8
:101C5000D8FBD9F9DCF781ADB17FE493A3C39A60D7
:101C6000028126DBDDB171600281267B08E493FAF4
:101C7000A3B152DBF87A30B152752200752300B15E
:101C800071EAFCEBFDC3ED94FE400EB1718A278B27
:101C900028ED30E0048A828B83B1717AC270D8C398
:101CA000ED94FE601050CEBD0022EC600675200061
:101CB0000200008100A827A9280809D804D90281B8
:101CC000C9B175EA89AAF281BB0D8199C3ED94036C
:101CD0005049EDA2E092007AC5C3E5829400E58305
:101CE000941C5093200010438F02438F0175B7A5B9
:101CF00075B7F1F030001FA827A9280809438F0104
:101D0000538FFDD804D902A11689AAE275B7A5752B
:101D1000B7F1F0A3A103538FFC81757AC1BD030C09
:101D2000E493A3FAB136DCF8B12E81758177AA224B
:101D3000AB23B152EBFAEA6222752608C3E52313FE
:101D4000F523E52213F52250066323A0632201D573
:101D500026EAB1BFB1BF75260AEAF4200102D28497
:101D6000300102C284B1BFC3134002C201D526EBC9
:101D700022B175EAFB208402A175308402A17A7534
:101D80002608AE24AF25C3EF13FFEE13FEB1C3B197
:101D9000BFC3EA133084024480FA30E703632201B0
:101DA000C3E52313F523E52213F52250066323A090
:101DB000632201D526D9E52265236523F52222AECB
:101DC00024AF250E0FDEFEDFFCD20122424C486517
:0A1DD0006C6934373132F33006013C
:00000001FF
